:100FD900121624300005C200120C93300A05C20A09
:100FE900121E3830030CC203200205121DF78002BD
:070FF900C202121F3180DC6F
:0506AA00011E00C10C5F
:1018590090E6BAE090E000F012008090E680E03077
:10186900E71300000090E6247402F0000000E49001
:10187900E625F08011000000E490E624F000000065
:1018890090E6257440F090E000E0600543B14080A7
:101899000353B1BFE490E6FBF090E60174EAF0204F
:0818A9000C04D20CD28CD322F6
:101EA60090E000E090E740F0E490E68AF090E68B60
:041EB60004F0D3223F
:0D1F040090E6BAE090E001F0120080D322D8
:101EBA0090E001E090E740F0E490E68AF090E68B4B
:041ECA0004F0D3222B
:051F5E00120080D322F7
:10017800E4F522F523F524F525F526F527F531F5DF
:1001880030F52FF52ED20590E6BBE0F52F90E6BDB1
:10019800E0F53090E6BCE0F53190E6BAE064A67090
:1001A8007190E6A0E04480F07F02121000782E12D1
:1001B8000B8BEF5403FFE48F1EAF31AE30AD2FAC85
:1001C8002E7802120B2B8F318E308D2F8C2EE51E40
:1001D8007016E53124FFFFE53034FFFEE52F34FFCC
:1001E800FDE52E34FFFC8008AF31AE30AD2FAC2ECC
:1001F8008F318E308D2F8C2EE51E70047F04800287
:10020800AF1E8F1E851E35AB31AD30AF2F121213C6
:10021800C1A890E6BAE0120BFA064A10064318067F
:100228003420062028061630061632062A380639E3
:1002380040063E50062F5206845606965802AC6871
:1002480002BC6C0651700651710651720651730654
:10025800517406517506517606517706667806661A
:100268007906667A06667B06667C06667D06667E85
:1002780006667F02B18802B68A02B18C02B68E0287
:10028800B19002B69202B19402B69602B19802B643
:100298009A02B19C02B69E0678A002BCA202BCA437
:1002A800000006A6121BEBC1A853807FC2053005CB
:1002B8000343808090E6BAE0F52DE5312401F5315D
:1002C800E43530F530E4352FF52FE4352EF52EE5FD
:1002D8002D2470700261B024FE700261B024FE709B
:1002E8000261B024FE700261B024F260062402604C
:1002F8000261B3E4F51CF51D90E68BF0121EF65072
:10030800267B007A0079251219BB501BAB25AA263B
:10031800A9271209DBF5289000011209F4F52990A4
:1003280000021209F4F52A90E6A0E04480F07F016B
:10033800121000E5315407FFE48F1EAF31AE30AD27
:100348002FAC2E7803120B2B8F318E308D2F8C2EE5
:10035800E51E7016E53124FFFFE53034FFFEE52F7A
:1003680034FFFDE52E34FFFC8008AF31AE30AD2FF1
:10037800AC2E8F318E308D2F8C2EE51E70047F08A9
:100388008002AF1E8F1EE58054C04408F580AF314F
:10039800AE30AD2FAC2EEC4D4E4F600AE5A054E0C8
:1003A8004408F5A08141813975220390E6A0E04414
:1003B80080F0E52270037522057F01121000E531F7
:1003C800540FFFE48F1EAF31AE30AD2FAC2E780442
:1003D800120B2B8F318E308D2F8C2EE51E7016E56B
:1003E8003124FFFFE53034FFFEE52F34FFFDE52E15
:1003F80034FFFC8008AF31AE30AD2FAC2E8F318E7C
:10040800308D2F8C2EE51E70047F108002AF1E8F5A
:100418001EE58054C04522F580AF31AE30AD2FAC1B
:100428002EEC4D4E4F600AE5A054E04410F5A08034
:1004380008E5A054E0451EF5A05380BFE52D120B3A
:10044800FA05CA6C05CA8805CA8A05CA8C05CA8E07
:10045800060990060992060994060996047A9804F2
:100468007A9A047A9C047A9E05CAA2047AA40000A7
:1004780006A8E52DB4A40A752B08752C08C20480BB
:1004880008752B05752C10D204121F43E531240181
:10049800F531E43530F530E4352FF52FE4352EF518
:1004A8002EE47F01FEFDFCAB31AA30A92FA82EC394
:1004B800120B1A7015438040E58054C0452BF58017
:1004C800E5A054E0451EF5A08010E58054C0452BFA
:1004D800F580E5A054E0452CF5A0121F52121E919C
:1004E800E58054C04407F580E5A054E04401F5A038
:1004F800A20492068523388524391219520524E569
:100508002470020523E53124FFF531E53034FFF589
:1005180030E52F34FFF52FE52E34FFF52E90E62534
:10052800E0702DB52408E523B4020330040DE5245A
:100538007004E52364017053300450E4FFFEFDFCB1
:10054800AB31AA30A92FA82ED3120B1A403D80290F
:10055800E52464404523700330040BE524642045FA
:10056800237028300425E4FFFEFDFCAB31AA30A936
:100578002FA82ED3120B1A4012A2049206852332FA
:100588008524331212C8E4F523F524E4FFFEFDFCAC
:10059800AB31AA30A92FA82ED3120B1A400281A979
:1005A800A2049206753800753900753A23851E3BFA
:1005B8001213B8A20492068523328524331212C876
:1005C800C1A8E4FFFEFDFCAB31AA30A92FA82ED3A9
:1005D800120B1A400C121F527B007A00792E121C43
:1005E800ACE5A054E0451EF5A0438040121E91E5FD
:1005F80026452745257002C1A8AB2AAD29AF28801A
:100608006A7B007A00792EAD1E121501C1A890E60A
:10061800BAE0FF121B0E805B90E6BCE0FF121F637E
:100628008051121ACF804C121908804712178D80FA
:1006380042121E4F803D1216A480387F18121A4AA3
:1006480080317F10121A4A802A30081290E6A0E002
:100658004480F07B007A00792E121800804290E6E0
:10066800BAE0FF90E6BCE0FDA3E0FB120EAB8030E1
:10067800121BB790E6A0E04480F0802490E6A0E04A
:100688004480F07B007A00792E121DAD801290E62E
:10069800A0E04480F0AF31AE301214618002C32272
:0206A800D3225B
:0A1F27000001020203030404050593
:0806AF00C101C100C103C10239
:10162400750A00750B907512007513A27508007584
:1016340009CC7510007511EC75140175154C750CF9
:1016440000750DAC750E01750F0C1218B1D2E8437C
:10165400D82090E668E0440BF090E65CE0443DF06E
:10166400D2EA00000090E660E04402F0121EE2902C
:10167400E6FB7402F090E600E054E5F090E60174B5
:101684000AF0121F11121F1CE490E672F075B65096
:10169400F5B1121723D204121C4FD202538EF82232
:091F3100300D05C20D121D5A22EB
:101E3800C28C90E600E054E7441054FDF0D204123E
:071E48001C4FD202021F3AF9
:101DF70053B1BF121DD220011690E682E030E704EE
:101E0700E020E1EF90E682E030E604E020E0E40243
:021E17001CD8D5
:100C930090E6B9E0B4B0091201785002C1AAC1A329
:100CA30090E6B9E0B40C004002C1A3900CB425E077
:100CB30073A146A1BAC1A3C137C1A3C1A381CCC14A
:100CC300A3A141A13CA132A13790E6BBE024FE6081
:100CD3002214603324FD601114602224067047E55A
:100CE3000A90E6B3F0E50B8037E51290E6B3F0E542
:100CF30013802DE50C90E6B3F0E50D8023E50E900F
:100D0300E6B3F0E50F801990E6BAE0FF121D04AADE
:100D130006A9077B01EA494B600CEE90E6B3F0EFBE
:100D230090E6B4F0A1B890E6A0E04401F0A1B812B7
:100D33001EBAA1B8121F04807C121859C19B121E3F
:100D4300A6C19B90E6B8E0247F600F1460132402D1
:100D5300705CA201E43325E08041E490E740F08039
:100D63003F90E6BCE0547EFF7E00E0D394807C009D
:100D730040047D0180027D00EC4EFEED4F2427F5FB
:100D830082741F3EF583E493FF3395E0FEEF24A1C5
:100D9300FFEE34E68F82F583E0540190E740F0E400
:100DA300A3F090E68AF090E68B7402F0800790E659
:100DB300A0E04401F0C19B90E6B8E024FE6011245A
:100DC30002706F90E6BAE0B40104C2018064805BF4
:100DD30090E6BAE0705590E6BCE0547EFF7E00E0FA
:100DE300D394807C0040047D0180027D00EC4EFEA4
:100DF300ED4F2427F582741F3EF583E493FF33956B
:100E0300E0FEEF24A1FFEE34E68F82F583E054FE8B
:100E1300F090E6BCE05480131313541FFFE0540F0B
:100E23002F90E683F0E04420F0800790E6A0E044B2
:100E330001F08064121F5E505F90E6B8E024FE600C
:100E43001C2402705390E6BAE0B40104D201804836
:100E530090E6BAE06402604090E6A0803790E6BC7A
:100E6300E0547EFF7E00E0D394807C0040047D014B
:100E730080027D00EC4EFEED4F2427F582741F3E69
:100E8300F583E493FF3395E0FEEF24A1FFEE34E610
:100E93008F82F583E04401F090E6A0E04480F022E5
:080EA30090E6A0E04401F022FA
:0D06B700C108C1090116000117000118005B
:10121300E490E6CEF000000090E6CFEFF00000008F
:1012230090E6D0EDF000000090E6D1EBF05380BFE4
:10123300121F4375360275370490E6D0E0FF90E63F
:10124300D1E04FFF90E6CFE04F605FE58054C044AC
:1012530009F580E5A054E04537F5A0E4F5BB121984
:10126300B33009D5E58054C0440AF580E5A054E0C5
:101273004401F5A090E6D17401F0000000E490E68B
:10128300D0F000000090E6CFF0D207121ECE90E619
:10129300D1E516F000000090E6D0E517F00000005D
:1012A30090E6CFE518F0C209808F8535374380403B
:1012B30090E6D17401F01536E5366002413C90E6C4
:0512C300487406F02252
:1019080090E6BCE064017039D20890E618E054FE15
:10191800F090E61AE054F7F000000090E6047480B6
:10192800F00000007406F0000000E4F07F03FE12EF
:10193800100090E6C2E04404F090E6C1E04401F0F3
:0A19480022C2081218B11217232260
:10178D0090E6BCE05402C43354E0FFE05401C4338E
:10179D00333354804FFFE0540433333354F84FFF49
:1017AD00E0540825E04FFFE05410C3134FFFE05401
:1017BD0020131313541F4FFFE05440C41354074F0D
:1017CD00FFE05480C413131354014F90E740F0E42D
:0A17DD0090E68AF090E68B04F022FB
:101E4F0090E74074B5F0A37403F0E490E68AF09045
:061E5F00E68B7402F02284
:101BB70090E6A0E04480F090E680E054FDF0E04439
:101BC70008F07FF47E01121A0490E65D74FFF0902E
:101BD700E65FF05391EF90E6FB7402F090E680E049
:041BE70054F7F0229D
:1016A40090E6BCE014601C146020146033240370C2
:1016B400599019B9E493FC74019390E740F0ECA3BA
:1016C400F0805090E74074FE804590E6BDE090E7DE
:1016D40040B40104740780027404F0E4A3F080337E
:1016E400E58054C0440DF580E5A054E04401F5A024
:1016F40090E6F1E090E740F090E6F2E090E740F009
:1017040090E6F0E090E741F0800990E7407405F03E
:0F171400A304F0E490E68AF090E68B7402F022D2
:101ACF00E58054C04402F580E5A054E04401F5A040
:101ADF0090E6F1E090E740F090E6F2E090E740F01A
:101AEF00121D5AEE90E74030E706E04440F08004C4
:0F1AFF00E054BFF0E490E68AF090E68B04F0220A
:1013B800300677E53BC3941040028160AB38AA3908
:1013C800A93A120A2124FFFDE5F034FFFCED25E0DF
:1013D800FFEC33FE74012FF58274F83EF583E0F5D7
:1013E8003C74002FF58274F83EF583E0F53DC37434
:1013F80010953BFFE53DAE3CA807088005CEC3131A
:10140800CE13D8F9F53D8E3CED25E0FFEC33FE74A4
:10141800002FF58274F83EF583E53DF074012FF551
:101428008274F83EF583E53CF022AB38AA39A93A34
:10143800AE02AF01EF4E6020120A2124FFF582743C
:10144800F735F0F583E0FFC37408953BFEEFA80677
:09145800088002C313D8FCF02245
:101501008D358B328A338934E4F536F537120B5138
:10151100E4FBFAF9F8C3120B1A503DE490E6CEF061
:10152100000000AB32AA33A9349000011209F490F3
:10153100E6CFF00000009000021209F490E6D0F02E
:101541000000009000031209F490E6D1F0000000C1
:101551001219B3D207121ECE00000090E6B0E0F5DA
:101561003700000090E6AFE0F536438040E5A05437
:10157100E04535F5A0D206E4F538F539121952D215
:1015810006753800753900753A3685353B1213B842
:0715910090E6487406F02209
:101B0E008F327F047E00121000E58054C04404F52D
:101B1E0080E5A054E04401F5A0E53224CE600B240C
:101B2E0002701790E6F07410800790E6BDE090E624
:0B1B3E00F0F090E6BCE090E6F1F02231
:100EAB008F328D338B34E4F538F537F536F53590D5
:100EBB00E6A0E04480F07E3C7F0E12112DE532243B
:100ECB008824F8500280055380C08008E58054C008
:100EDB004406F580E5322490B410005039900EF2A0
:100EEB0025E05002058373E112E112E11CE11CE1E4
:100EFB0012E112E11CE11CE112E112E11CE11CE127
:100F0B0012E112E11CE11CE580547F4440F5808026
:100F1B00084380C0800353807FE4853438F537F570
:100F2B0036F535AF38AE37AD36AC357808120B3EEB
:100F3B00EEFAE533F538EAF537E4F536F535E5380D
:100F4B002401F538E43EF537E43536F536E435352E
:100F5B00F535E4FFFE7D01FCAB38AA37A936A83581
:100F6B00C3120B1A700A7538FF7537FFF536F53556
:100F7B001219B3AF38AE37AD36AC357808120B2B30
:100F8B0090E6F0EFF090E6F1E538F01219B3E532A8
:100F9B0064796029E532647B6023E532647D601DF2
:100FAB00E532647F6017E53264716011E53264737A
:100FBB00600BE53264756005E532B4771090E7405D
:0E0FCB00E532F0E490E68AF090E68B04F02226
:101BEB007F047E00121000E58054C04401F580E5AF
:101BFB00A054E0FF90E6BCE0044FF5A01219B3E44B
:101C0B0090E6F0F090E6BDE090E6F1F090E6A0E013
:041C1B004480F022EF
:101A4A008F32851F337F14121F637F047E001210AA
:101A5A0000E58054C04410F580E5A054E04403F545
:101A6A00A0E490E6F0F0E532B4180890E6F17401CB
:101A7A00F0800AE532B41005E490E6F1F0AF3312D3
:051A8A001F630219B307
:1006C400011F11033E000000034100000003440029
:0706D40000000347000000D5
:1017230090E6F574FFF090E6F374A0F0E490E6C35E
:10173300F090E6C1E054FEF090E6C27402F090E649
:10174300C0744EF075AF077E3B7F7C12112D7E3B3C
:101753007FCC12112D7F02121000000000E490E6EE
:10176300C4F000000090E6C5F090E6C6F090E6C72E
:10177300F090E6C8F090E6C9F090E6CAF090E6CBA8
:0A178300F090E6CCF090E6CDF022E5
:0619B300E5BB30E7FB225A
:101E9100000000E490E6D0F000000090E6D104F0EC
:051EA100C207021ECE85
:1019520030061C000000E490E6CFF000000090E6A4
:10196200D0F000000090E6D104F0D207021ECE9023
:10197200E6F1E0FF74002539F58274F83538F58315
:10198200EFF01219B390E6F0E0FF74002539F5820A
:0919920074F83538F583EFF022FA
:101ECE000000002007047F0080027F068FBB000009
:041EDE00000219B332
:101CAC000000009000031209F490E6D1F00000004F
:101CBC009000021209F490E6D0F0000000900001B0
:0C1CCC001209F490E6CFF0C207021ECE11
:041C7E00AF3AAE3992
:101C8200AD07AC06ED2401FBE43CF59AAF03EFF59A
:101C92009B759DE48D828C83E0F59E7F0190E67BAF
:0A1CA200E090E67CF00FBF21F42271
:10100000EF24FE607614700201EC14700201F324E8
:10101000036002212CE51F24F0601F146029146076
:101020003314603D14604724F46002212C7E3B7F22
:101030005B12112D7E3D7F5A01F07E3B7F11121114
:101040002D7E3D7F1601F07E3B7F3A12112D7E3DB5
:101050007F3901F07E3A7FF012112D7E3C7FF50141
:10106000F07E3C7FB312112D7E3C7F2F01F07E3C41
:101070007FD412112D7E3C7F5080757E3C7F711293
:10108000112D7E3C7F9212112DE51F24F060181463
:10109000602214602C14603614604024F460022135
:1010A0002C7E3B7FA38049903B9FE090E461F090D1
:1010B0003BA08032903BA1E090E461F0903BA280A5
:1010C00025903B9DE090E461F0903B9E8018903D20
:1010D00037E090E461F0903D38800B903AEEE0907C
:1010E000E461F0903AEFE090E462F0227E3B7FED25
:1010F00002112D7E3B7FCC12112DE51F24EC7008D0
:1011000075343B753532800675343B7535C4E4FF64
:10111000E5352FF582E43534F583E0FE74202FF5B4
:0D11200082E434E4F583EEF00FBF08E42212
:10112D008E398F3A8F828E83E024E0604224E06016
:10113D006E24E0700221DC246060024112783E864C
:10114D000308E6FA08E6F9EB8A838982AA39A93AF7
:10115D007B016401700AE53A65827004E5396583A7
:10116D0070024112121C7EAA39A93A783E410A78C2
:10117D0041860308E6FA08E6F9EB8A838982AA39E3
:10118D00A93A7B016401700AE53A65827004E5397C
:10119D0065836071121C7EAA39A93A7841805E7808
:1011AD0044860308E6FA08E6F9EB8A838982AA39B0
:1011BD00A93A7B016401700AE53A65827004E5394C
:1011CD0065836041121C7EAA39A93A7844802E7835
:1011DD0047860308E6FA08E6F9EB8A838982AA397D
:1011ED00A93A7B016401700AE53A65827004E5391C
:1011FD0065836011121C7EAA39A93A7847760108D9
:06120D00A60208A6012262
:031F63008F1F22AB
:0406DB00021C0000FD
:1018B10000000090E6047480F00000007402F00063
:1018C10000007406F0000000E4F090E614E0440823
:1018D100F0E054FCF0E04402F090E612E054F4F041
:1018E10090E615E0547FF090E613E0547FF000009D
:1018F1000090E6187405F00000007415F000000077
:0719010090E61A7409F022C0
:101D8400E4FFFE90E68BE07012C3EF9410EE6480E3
:101D940094A750070FBF00010E80E8C3EF9410EE24
:091DA400648094A7400122D322BF
:0E1EF60090E6BEE07002A3E06002D322C32299
:101D3000121EF6500C90E68BE07006121D844001D6
:101D400022E51D2403FFE4351CFE90E68BE0FDD365
:0A1D5000EF9DEE9400500122C32223
:1019BB008B328A338934121D3050277440251DF920
:1019CB00E434E7FA7B01C003C002C001AB32AA3397
:1019DB00A934120BAB7403251DF51DE4351CF51C46
:1019EB00D3227B007A007900C003C002C001AB3266
:0919FB00AA33A934120BABC3227C
:1012C80030060890E6487406F0802BE53330E014C9
:1012D8002400F58274F83532F583E4F00533E533FC
:1012E80070020532000000E53290E698F000000038
:0812F80090E699E533F0D322E2
:081F430090E6A7E020E1F9227D
:061F5200121F430219B347
:1000800090E6837402F07422F07416F07436F02255
:0B1F1100E490E670F075B2FFF580224E
:0B1F1C00E490E671F075B41FF5A02200
:1017E700C0E0C083C082D2035391EF90E65D7408D6
:0817F700F0D082D083D0E03273
:10199B00C0E0C083C082D2005391EF90E65D74012A
:0819AB00F0D082D083D0E032BD
:101E6500C0E0C083C0825391EF90E65D7404F0D06A
:061E750082D083D0E032B0
:101E7B00C0E0C083C0825391EF90E65D7402F0D056
:061E8B0082D083D0E0329A
:101B4900C0E0C083C08290E680E030E70E85080CD3
:101B590085090D750E01750F0C800C750C00750D3E
:101B6900EC750E01750F2C5391EF90E65D7410F032
:071B7900D082D083D0E032DE
:101B8000C0E0C083C08290E680E030E70E85080C9C
:101B900085090D750E01750F0C800C750C00750D07
:101BA000EC750E01750F2C5391EF90E65D7420F0EB
:071BB000D082D083D0E032A7
:0117FF0032B7
:011F66003248
:011F67003247
:011F68003246
:011F69003245
:011F6A003244
:011F6B003243
:011F6C003242
:011F6D003241
:011F6E003240
:011F6F00323F
:011F7000323E
:011F7100323D
:011F7200323C
:011F7300323B
:011F7400323A
:011F75003239
:011F76003238
:011F77003237
:011F78003236
:011F79003235
:011F7A003234
:011F7B003233
:011F7C003232
:011F7D003231
:011F7E003230
:011F7F00322F
:011F8000322E
:011F8100322D
:011F8200322C
:011F8300322B
:011F8400322A
:011F85003229
:011F86003228
:011F87003227
:101C1F00C0E0C083C0825391BF90E6617402F09020
:101C2F00E6D1E0F51690E6D0E0F51790E6CFE0F5B7
:101C3F001890E6F574FFF0D209D082D083D0E0324D
:03000B00021A8F47
:101A8F00C0E0C0D0E51B14600904702FC28CD20BCC
:101A9F008029C28C758A00758C00C3E51A9428E5DD
:101AAF001964809480500C051AE51A70020519D23A
:101ABF008C8008D20A751900751A00D0D0D0E03288
:03003300021F4B5E
:071F4B0043B14053D8EF320F
:03005B00021F5829
:061F580053917FD20D320F
:101DAD008B328A338934120B51EF2401FFE43EFE4E
:101DBD00E43DFDE43CFC120B71121F43AB32AA3320
:051DCD00A934021CAC6A
:101461008E328F33E4F536F53790E624E0F534908B
:10147100E625E0F5350533E53370020532E532C383
:1014810013F532E53313F533121F4390E6D174029D
:10149100F0E5331533AE32700215324E6052E5A0DD
:1014A1005440FF0537E537AC367002053614240089
:1014B100F58274F83CF583EFF000000090E6D474F7
:1014C100FFF000000090E6D17402F0E537B535C1B8
:1014D100E536B534BC90E698F0000000E53790E6BB
:1014E10099F0E4F536F53790E6A5E030E3A380F70F
:1014F100E53690E698F0000000E53790E699F02295
:101800008B328A338934120B51E47BFF7AFFF9F86B
:10181000120A88AE02AF03E4FD121E19AB32AA33DE
:10182000A934120B51E47BFF7AFFF9F8D3120B1A9B
:101830005026E4FD74FFFFFE121E19AB32AA33A935
:1018400034120B51EF2401FFE43EFEED34FFFDECBA
:0918500034FFFC120B7180C4226C
:1006DF0060213B5B60010101012B01010702020256
:1006EF0002030602020100030203020202000000DD
:1006FF00000000003F60213B116002020202013343
:10070F0002070202020202030602010003020303B0
:10071F000202000000000000003F60213B3A60042D
:10072F000404040333040702020202020306020157
:10073F0000030203030202000000000000003F60FC
:10074F00213AF06001010808073301070202020293
:10075F00020306020100030203030202000000006D
:10076F000000003F60213CB360101010100F3310D9
:10077F000702020202020306020100030203030240
:10078F0002000000000000003F60213CD4602020E8
:10079F0020201F3320070202020202030602010279
:1007AF00030203030202000000000000003F60216B
:1007BF003D5A400101010101320107000000000014
:1007CF000102000100030203020302000000000007
:1007DF0000003F60213D1640020202020133020772
:1007EF0000000000000102000100030203030202E7
:1007FF00000000000000003F60213D394004040468
:10080F00040333040700000000000102000100038D
:10081F000203030202000000000000003F60213CC1
:10082F00F54008080808073308070000000000011A
:10083F000200010003020303020200000000000097
:10084F00003F60213C2F40101010100F3310070095
:10085F000000000001020001000302030302020076
:10086F000000000000003F60213C5040202020206D
:10087F001F332007000000000001020001000302E7
:10088F0003030202000000000000003F60213C0E45
:10089F00202020201F3A0101070202020203020258
:1008AF000201000302020202020000000000000029
:1008BF003F60213BCC20040404032A0403070602F3
:1008CF0002020302020201000302020302020000FD
:1008DF0000000000003F483BC4040404032A040343
:1008EF0007483B322020201F2A201F0760213B7C16
:1008FF0000040404032A040307060202020302028F
:10090F0002010003020203020200000000000000C7
:10091F003F60213C7160010000212F01B7070202E7
:10092F000203071203020003020202020202000086
:10093F0000120900123F423B9F0201423BA10403F8
:10094F00423B9D0807423D37100F423AEE201F6091
:10095F00213BA3600101192701AF01070202030721
:10096F001203000200030202020200020000120939
:10097F000012003F60213C92400101012201020759
:10098F000700000001020001000100030203020240
:10099F0002000000000000093F60213BED600101F3
:1009AF00010101010107020202020202060206060C
:0E09BF00060606060602000000000000003FCB
:0B09CD00011B01C10BC10A021900014F
:101EE200C2AFC28CE4F58E5389F0438901C2B9D2E4
:041EF200A9D2AF22A0
:101E1900C2AFC28C8D1BC20BC3E49FFDE49EFCEDD7
:0F1E2900F58AECF58CD2A9D2AFD28C300BFD220A
:0209D800C10D4F
:091F3A00C2AFC2FBD2EBD2AF2210
:101D5A00E58054C0440CF580E5A054E04401F5A0A8
:101D6A0090E6F1E0F53290E6F0E0F53290E6F2E046
:0A1D7A00F5335380C0AE32AF3322C0
:100090001201000200000040FD0308000000010200
:1000A00000010A06000200000040050009022000CD
:1000B00001010080960904000002FF00000007050E
:1000C00002024000000705860240000009022000ED
:1000D00001020080960904000002FF0000000705ED
:1000E0000202000200070586020002000902200049
:1000F00001030080960904000002FF0000000705CC
:1001000002024000000705860240000009072000A7
:1001100001040080960904000002FF0000000705AA
:100120000202400000070586024000000907200087
:1001300001050080960904000002FF000000070589
:1001400002020002000705860200020004030904FF
:100150001003580049004C0049004E005800200090
:100160001603580049004C0049004E00580020007A
:08017000200020002000000027
:101CD80090E682E030E004E020E60B90E682E03017
:101CE800E119E030E71590E680E04401F07F147ECA
:0C1CF80000121A0490E680E054FEF02276
:101DD20090E682E044C0F090E681F0438701000083
:041DE20000000022DB
:101C4F0030040990E680E0440AF0800790E680E0D7
:101C5F004408F07FDC7E05121A0490E65D74FFF0F5
:0F1C6F0090E65FF05391EF90E680E054F7F0229B
:101A04008E328F3390E600E054187012E5332401CF
:101A1400FFE43532C313F532EF13F533801590E646
:101A240000E05418FFBF100BE53325E0F533E53231
:101A340033F532E5331533AE32700215324E60059C
:061A4400121DE680EE22F7
:021D0400A9072D
:101D0600AE14AF158F828E83A3E064037017AD0106
:101D160019ED7001228F828E83E07C002FFDEC3E50
:091D2600FEAF0580DF7E007F00A6
:011D2F002291
:101DE6007400F58690FDA57C05A3E582458370F910
:011DF60022CA
:03004300021300A5
:0300530002130095
:1013000002199B00021E7B00021E65000217E70007
:10131000021B4900021B80000217FF00021F66002B
:10132000021F6700021F6800021F6900021F6A0097
:10133000021F6B00021F6C00021F6D00021F6E0077
:10134000021F6F00021F6600021F7000021F710063
:10135000021F7200021F7300021F7400021F75003B
:10136000021F7600021F6600021F6600021F660051
:10137000021F7700021F7800021F7900021F7A0007
:10138000021F7B00021F7C00021F7D00021F7E00E7
:10139000021F7F00021F8000021F8100021F8200C7
:1013A000021F8300021F8400021F8500021F8600A7
:0813B000021F8700021C1F0050
:0219B90007D64F
:030000000215984E
:0C159800787FE4F6D8FD7581490215DF6C
:1009DB00BB010689828A83E0225002E722BBFE021A
:0909EB00E32289828A83E493224D
:1009F400BB010CE58229F582E5833AF583E02250B8
:100A040006E92582F8E622BBFE06E92582F8E22201
:0D0A1400E58229F582E5833AF583E493221B
:100A2100BB010A89828A83E0F5F0A3E022500687A0
:100A3100F009E71922BBFE07E3F5F009E319228962
:0B0A4100828A83E493F5F07401932295
:100A4C0075F008758200EF2FFFEE33FECD33CDCC61
:100A5C0033CCC58233C5829BED9AEC99E5829840E4
:100A6C000CF582EE9BFEED9AFDEC99FC0FD5F0D6C1
:100A7C00E4CEFBE4CDFAE4CCF9A88222B800C1B9EB
:100A8C000059BA002DEC8BF084CFCECDFCE5F0CB29
:100A9C00F97818EF2FFFEE33FEED33FDEC33FCEB62
:100AAC0033FB10D703994004EB99FB0FD8E5E4F91D
:100ABC00FA227818EF2FFFEE33FEED33FDEC33FC0A
:100ACC00C933C910D7059BE99A4007EC9BFCE99AFE
:100ADC00F90FD8E0E4C9FAE4CCFB2275F010EF2F43
:100AEC00FFEE33FEED33FDCC33CCC833C810D70743
:100AFC009BEC9AE899400AED9BFDEC9AFCE899F87E
:0E0B0C000FD5F0DAE4CDFBE4CCFAE4C8F92210
:100B1A00EB9FF5F0EA9E42F0E99D42F0E89C45F031
:010B2A0022A8
:100B2B00E8600FECC313FCED13FDEE13FEEF13FFA8
:030B3B00D8F122CC
:100B3E00E8600FEFC333FFEE33FEED33FDEC33FC15
:030B4E00D8F122B9
:100B5100BB010789828A83020C2C5005E9F8020C3B
:100B610020BBFE05E9F8020C3889828A83020C4415
:100B7100BB010789828A83020C605005E9F8020CE7
:0A0B810054BBFE05E9F8020C6C22DB
:100B8B007401FF3395E0FEFDFC080808E62FFFF625
:100B9B0018E63EFEF618E63DFDF618E63CFCF6229E
:100BAB00BB011A89828A83D0F0D0E0F8D0E0F9D06B
:100BBB00E0FAD0E0FBE8C0E0C0F0020C815016E98F
:100BCB00F8D083D082D0E0F9D0E0FAD0E0FBC0823D
:100BDB00C083020C78BBFE16E9F8D083D082D0E03C
:0F0BEB00F9D0E0FAD0E0FBC082C083020C8A226E
:100BFA00D083D082F8E4937012740193700DA3A38A
:100C0A0093F8740193F5828883E47374029368609D
:060C1A00EFA3A3A380DF9D
:1015A400020FD9E493A3F8E493A34003F68001F275
:1015B40008DFF48029E493A3F85407240CC8C33348
:1015C400C4540F4420C8834004F456800146F6DF17
:1015D400E4800B01020408102040809006AAE47EF7
:1015E400019360BCA3FF543F30E509541FFEE4930C
:1015F400A360010ECF54C025E060A840B8E493A3D3
:10160400FAE493A3F8E493A3C8C582C8CAC583CAFD
:10161400F0A3C8C582C8CAC583CADFE9DEE780BEB5
:0109DA00001C
:0C0C2000E6FC08E6FD08E6FE08E6FF2200
:0C0C2C00E0FCA3E0FDA3E0FEA3E0FF223B
:0C0C3800E2FC08E2FD08E2FE08E2FF22F8
:100C4400E493FC740193FD740293FE740393FF22F6
:0C0C5400ECF608EDF608EEF608EFF622CC
:0C0C6000ECF0A3EDF0A3EEF0A3EFF02207
:0C0C6C00ECF208EDF208EEF208EFF222C4
:090C7800EBF608EAF608E9F622A1
:090C8100EBF0A3EAF0A3E9F02274
:090C8A00EBF208EAF208E9F2229B
:00000001FF
